:020000040000FA
:10000000831603138312031309308E2141285F30B6
:100010009C21A221E03EA200031C2028F43E0318EC
:1000200020288A0122088207AD280728AD28AD289C
:10003000272927298928072881288528072885280E
:100040002208DF3EA200031C0728F93E03180728F8
:100050008A0122088207322841285A2807280728BF
:1000600007287C284D309C2141309C2131309C2137
:100070002D309C2132309C210D309C210A309C2156
:10008000072883160313061286118312031306161C
:1000900086150530882183160313061786178616E2
:1000A00006148312031386110530882106120130CD
:1000B0008821072883120313061601308021861534
:1000C0000530882183160313861306138612061043
:1000D000831203138613061386120610053080213F
:1000E000831203130612000000000000000000004D
:1000F000861105308821072806160A30802106124D
:1001000007288B201930802107288B203C30802144
:1001100007288B20072883120313861322188617BB
:10012000061706138613A2188617061706138613DA
:1001300022198617061706138613A21986170617A3
:1001400006138613221A8617061706138613A21A99
:100150008617061706138613080083120313A221BD
:10016000A300A221A40086132218861706170613DF
:100170008613A218861706170613861322198617E8
:10018000061706138613A219861706170613861379
:10019000221A8617061706138613A21A8617061741
:1001A00006130000000000000000861323188617C5
:1001B000061706138613A318861706170613861349
:1001C00023198617061706138613A3198617061711
:1001D00006138613231A8617061706138613A31A07
:1001E0008617061706138613231B86170617061392
:1001F0008613A31B86170617061386132418861763
:10020000061706138613A4188617061706138613F7
:1002100024198617061706138613A41986170617BE
:1002200006138613241A8617061706138613A41AB4
:100230008617061706138613241B86170617061340
:100240008613A41B861706170613861307288B2010
:10025000A301A4010617061383160313861783123E
:10026000031306170613861BA31406170613861B13
:10027000231506170613861BA31506170613861BE0
:10028000231606170613861BA31606170613861BCE
:10029000231706170613861BA31706170613861BBC
:1002A000241406170613861BA41406170613861BB0
:1002B000241506170613861BA41506170613861B9E
:1002C000241606170613861BA41606170613861B8C
:1002D00024170617061383160313861383120313BA
:1002E00023089C2124089C210728A0000B30FF3EF6
:1002F000031D7729000000000000A00B76290800EC
:10030000A0007D30FF3E031D8229A00B812908003B
:10031000A10064308021A10B8929080083160313F2
:100320008614061183160313181599009816831264
:100330000313981718160800831203130C1E9E2926
:1003400099000800831203138C1EA4291A080800C0
:02400E00423F2F
:00000001FF
